:1000000063C0000088C0000086C0000084C00000FB
:1000100082C0000080C000007EC000007CC00000E4
:100020007AC0000078C0000076C0000074C00000F4
:1000300072C0000070C000006EC000006CC0000004
:100040000C94BF0E68C000000C94080D0C94420D77
:1000500062C000000C94C9105EC000005CC00000CB
:100060005AC0000058C00000000000070002010054
:100070000003040600000000000000000102040864
:100080001020408001020408102001020408102002
:10009000040404040404040402020202020203032E
:1000A00003030303000000002300260029000000D2
:1000B0000000250028002B0000000000240027007D
:1000C0002A005908FC0DF81011241FBECFEFD8E00C
:1000D000DEBFCDBF11E0A0E0B1E0E8E6F3E202C090
:1000E00005900D92A834B107D9F723E0A8E4B1E058
:1000F00001C01D92A134B207E1F710E0C8ECD0E0D6
:1001000004C02297FE010E94A211C23CD107C9F788
:10011000CCD70C94FF1074CF0895089508950895D6
:1001200008950895089508950895089508950895E7
:10013000089508952F923F924F925F926F927F920F
:100140008F929F92AF92BF92CF92DF92EF92FF92E7
:100150000F931F93CF93DF93CDB7DEB727970FB6DB
:10016000F894DEBF0FBECDBF8F83862FDA0160E02B
:1001700070E0412C512C32014A94A12CB12C650124
:10018000E12CF12C8701EA9420E030E0A901E82F6E
:10019000F0E0FE83ED833197FA83E983FF812F2E10
:1001A000312C8D819E810A969C838B8339C0FB0103
:1001B000EE0FFF1FEA0FFB1F808091802814390487
:1001C00068F1FB013196EE0FFF1FEA0FFB1F019054
:1001D000F081E02DE215F30508F17F0100E010E069
:1001E000940140E050E08D819E81860F971FBC01F5
:1001F0006F5F7F4F660F771F6A0F7B1FFB01408089
:100200005180612C712CFC01EE0FFF1FEA0FFB1FC8
:10021000A080B180C12CD12C6B817C816F5F7F4F1E
:1002200089819A816817790714F2EF816E2F70E047
:1002300080E090E07F926F925F924F920E947A0EE0
:100240000F900F900F900F9027960FB6F894DEBF87
:100250000FBECDBFDF91CF911F910F91FF90EF9017
:10026000DF90CF90BF90AF909F908F907F906F90D6
:100270005F904F903F902F9008950E94090F6093D8
:100280004F0170935001809351019093520181E08E
:1002900080935301089580937501E0917301F0E01C
:1002A000DF01A459BE4F9C91911103C0837051F49A
:1002B000E4CFEE0FFF1FEE0FFF1FEC5AFE4F8381BE
:1002C00084FDF6CF0895E7CFBF92CF92DF92EF92F1
:1002D000FF920F931F93CF93DF934CE6C42E41E020
:1002E000D42E56E7E52E51E0F52E04E511E0B12CB1
:1002F000D601ED916D01F0E0EB5CFE4F40816B2D7E
:1003000086E392E0FCD686E392E0E0D6C0E0D0E05F
:10031000F801EC0FFD1F20814C2F6B2D86E392E03E
:10032000F2D62196C430D10599F786E392E0CED675
:10033000C0E0D0E04C2F6B2D86E392E0D4D6F701DD
:10034000EC0FFD1F40816B2D86E392E0D0D6219605
:10035000C032D10579F786E392E0B8D6B394B0E223
:10036000EB0EF11C0C5F1F4F86E0B812C1CF6091FD
:100370007301E62FF0E0E459FE4FE081F0E0EB5C22
:10038000FE4F408186E392E0DF91CF911F910F9164
:10039000FF90EF90DF90CF90BF90B1C64F925F92E9
:1003A0006F927F928F929F92AF92BF92CF92DF9285
:1003B000EF92FF920F931F93CF93DF932FEF829FC4
:1003C000C001112406E711E07C013EE1E30EF11CBF
:1003D0006CE6A62E61E0B62E6C01E8E1CE0ED11CD3
:1003E000C4E5D1E03C016C1A7D0A38C0FE01E40D81
:1003F000F51DB201680D791D408186E792E05FD658
:10040000FFEF4F1A5F0A24E04216510479F7F50115
:1004100041915F01B60186E792E051D6812C912C83
:10042000F801E80DF91DB4016E0D7F1D408186E7CE
:1004300092E045D6FFEF8F1A9F0A20E282169104C0
:1004400079F7005E1F4F30E2E30EF11C8FEFC81A00
:10045000D80A2496E2E006331E0731F043018C0EE1
:100460009D1E412C512CC2CFDF91CF911F910F9136
:10047000FF90EF90DF90CF90BF90AF909F908F90C4
:100480007F906F905F904F9008954F925F926F9220
:100490007F928F929F92AF92BF92CF92DF92EF9214
:1004A000FF920F931F93CF93DF9380934E012FEF13
:1004B000829FC00111247C013EE1E30EF11C06E79E
:1004C00011E06C01E8E1CE0ED11C7CE6A72E71E0B4
:1004D000B72EC4E5D1E04C018C1A9D0A38C0B20198
:1004E000660D771D86E792E0E7D5FE01E40DF51D68
:1004F0008083FFEF4F1A5F0A24E04216510479F718
:10050000B60186E792E0D8D5F50181935F01612CB1
:10051000712CB3016E0D7F1D86E792E0CDD5F801F9
:10052000E60DF71D8083FFEF6F1A7F0A20E2621647
:10053000710479F730E2E30EF11C005E1F4F8FEF7C
:10054000C81AD80A2496E2E006331E0731F03401B7
:100550006C0E7D1E412C512CC2CF88E592E0DF91BC
:10056000CF911F910F91FF90EF90DF90CF90BF90B0
:10057000AF909F908F907F906F905F904F90EAC761
:10058000EF92FF920F931F93CF93DF93E12C18EC20
:1005900000E6FF24F3948E2D78DFE7E5F1E0ACE68A
:1005A000B1E046E751E010C0EA01C20FD31F188244
:1005B0002F5F3F4F20323105B9F73496405E5F4FD1
:1005C00081E0EF36F80771F0EF0123971883EF0110
:1005D00022971882EF01219718820083FD9220E074
:1005E00030E0E2CF8E2DDADEE39483E0E812D3CF61
:1005F00047E06CEF73E086E792E061D540E36DEF92
:1006000073E086E792E05BD543E66EEF73E086E742
:1006100092E0DF91CF911F910F91FF90EF904FC526
:1006200060E088E592E00E94240C882371F061E08C
:1006300088E592E00E94240C882339F062E088E586
:1006400092E00E94240C811116C06CEF73E086E7E3
:1006500092E032D5873089F46DEF73E086E792E05F
:100660002BD5803351F46EEF73E086E792E024D50A
:10067000833619F4089584DFE8CF82CF60E076E90D
:1006800086E392E020D56CE870E086E392E014D631
:1006900063E671E086E392E013D66DE870E086E3EE
:1006A00092E012D66EE870E086E392E011D66FE831
:1006B00070E086E392E010D660E970E086E392E0B5
:1006C0000FD661E970E086E392E00ED662E970E051
:1006D00086E392E00DD663E970E086E392E00CD603
:1006E00064E970E086E392E00BD665E970E086E3AA
:1006F00092E00AD666E970E086E392E009D667E9FF
:1007000070E086E392E008D668E970E086E392E064
:1007100007D669E970E086E392E006D660E088E5F6
:1007200092E00E94FF0B61E089E00E94271061E0E7
:100730008AE00E94271088E592E00E94F50B88E588
:1007400092E00E94F50B88E592E00E94F50B88E5A7
:1007500092E00E94F50B88E592E0FCD661DF80E034
:1007600094DE68EC70E080E090E007C086E392E001
:10077000D3D46AE070E080E090E00E94450F86E309
:1007800092E0A4D46091730186E392E0A7D48AE753
:1007900092E00E946D0C892B49F396DD88E592E08A
:1007A000D9C6CF938091730180937201C0E06C2F02
:1007B00088E592E00E942E0C882341F0909174010C
:1007C000892F880F890F8C0F80937301CF5FC330FF
:1007D00071F763E088E592E00E942E0C8823F9F01F
:1007E00063E088E592E00E94420C63E088E592E0D5
:1007F0000E94630C91E0811101C090E0909374011C
:1008000080917301911106C063E00E9426119093BC
:10081000730105C0833018F48D5F8093730163E02A
:1008200088E592E00E94630C91E0811101C090E0A4
:10083000909374019091730180917201981761F007
:1008400088E592E087D66091730186E392E046D412
:1008500086E392E0CF913AC4CF9108951F93CF934E
:10086000DF9366E088E592E0EFD7882309F495C02E
:100870008091730190E0FC01E459FE4F208121300A
:1008800009F452C060F1223009F0A0C0FC01EE0F63
:10089000FF1FEE0FFF1FEC5AFE4F4381417060E0D7
:1008A00088E592E0C3D6E091730184E0E89FF0010F
:1008B0001124EC5AFE4F438142FB442740F961E08A
:1008C00088E592E0B3D6E091730184E0E89FF001FF
:1008D0001124EC5AFE4F43814695417057C0FC01EC
:1008E000EE0FFF1FEE0FFF1FEC5AFE4F438146FB3A
:1008F000442740F960E088E592E098D661E088E519
:1009000092E0A2D7482F61E088E592E08FD6E0918F
:10091000730184E0E89FF0011124EC5AFE4F4381FB
:10092000441F4427441F32C0FC01EE0FFF1FEE0F8F
:10093000FF1FEC5AFE4F43814295417060E088E50D
:1009400092E074D6E091730184E0E89FF0011124F5
:10095000EC5AFE4F838183FF08C041E061E088E5E7
:1009600092E064D640E060E002C040E061E088E5EB
:1009700092E05CD6E091730184E0E89FF0011124DD
:10098000EC5AFE4F438145FB442740F962E088E57D
:1009900092E0DF91CF911F9149C6C0E0D0E013E013
:1009A00080917301612F0E942611692F892F90E099
:1009B0008C179D0711F441E002C040E06C2F88E5E0
:1009C00092E034D62196C330D10551F7DF91CF9113
:1009D0001F910895CF93DF9366E088E592E034D7C6
:1009E0008823D1F065E088E592E038D7882331F09C
:1009F00080914E01D3DC81E080934D0164E088E575
:100A000092E02CD7882341F06091730186E392E055
:100A100060D381E080934D0164E088E592E014D7D3
:100A2000811105C080914D01811118C025C0C0E021
:100A3000D1E06C2F88E592E011D7882359F0D0934C
:100A40004D0180914E01AADC8C2F1FDD3DDC88E535
:100A500092E080D5CF5FC33061F7E4CFC0E0D0E053
:100A60006C2F88E592E0F0D6D80FCF5FC730C1F782
:100A7000D11102C010924D01DF91CF9108958617D8
:100A8000970744F0841795075CF04617570744F022
:100A900081E00895481759071CF064177507C4F7DB
:100AA00080E00895CF92DF92FF920F931F93CF9330
:100AB000DF931F92CDB7DEB766E088E592E0C4D63B
:100AC000882311F160E088E592E03AD5882321F08F
:100AD00060E088E592E043D560E088E592E026D5C5
:100AE00081118BC060E088E592E04BD595958795A4
:100AF0009595879546E051E065E080951BDB709306
:100B000005016093040179C0C12CD12CFC2C6C2D03
:100B100088E592E00BD5882351F16C2D88E592E0B1
:100B20000FD5811165C080917301F60194E0899F12
:100B3000E00DF11D1124EC5AFE4F40816C2D88E52B
:100B400092E0498327D58C016C2D88E592E019D578
:100B5000B8017595679575956795498150E09595AC
:100B60008795959587958BDF811142C038C000919C
:100B7000730110E06C2D88E592E003D5F801EE0FCB
:100B8000FF1FEE0FFF1FEC0DFD1DEC5AFE4F95955C
:100B900087959595879580836C2D88E592E0F1D4B3
:100BA0008C016C2D88E592E0F5D415950795159587
:100BB000079595958795959587950817190779F065
:100BC0006C2D88E592E0DDD49C013595279535950F
:100BD00027954C2D6091730186E392E094D2EFEF5C
:100BE000CE1ADE0AF3E0CF16D10409F08FCF05C08C
:100BF0006F2D88E592E0B3D4F2CF0F90DF91CF91C3
:100C00001F910F91FF90DF90CF9008950F931F9346
:100C1000CF93DF93E0917301F0E0E459FE4F8081C0
:100C2000813009F4A7C020F0823009F062C1FCC015
:100C300065E088E592E008D6882349F100917301C8
:100C400010E0C0917501D0E060E088E592E099D4B1
:100C5000F801A5E0EE0FFF1FAA95E1F7EC0FFD1FCD
:100C6000EA58FE4F95958795959587958083609175
:100C700073018091750120E2629FF0011124E80F59
:100C8000F11DEA58FE4F408186E392E034D265E0E0
:100C900088E592E0EDD5882339F0409175016091A7
:100CA000730186E392E01FD266E088E592E0CCD53E
:100CB000882309F41EC160E088E592E0CFD588233F
:100CC000C1F06091730124E0629FC0011124FC0116
:100CD000EC5AFE4F238126FD02C0206401C02F7B09
:100CE0002383FC01EC5AFE4F238143E086E392E02C
:100CF0000AD261E088E592E0B1D5811107C062E0D7
:100D000088E592E0ABD5811125C0F3C0C0E0D0E00A
:100D100060917301FE0180E2689FE00DF11D1124D6
:100D2000EA58FE4F10824C2F86E392E0DCD16091AE
:100D30007301FE0190E2699FE00DF11D1124EA5854
:100D4000FE4F408186E392E0D2D12196C032D10598
:100D5000F9F6D5CF6091730124E0629FC0011124A0
:100D6000FC01EC5AFE4F238127FD02C02068B4C06D
:100D70002F77B2C066E088E592E066D5882309F453
:100D8000B8C060E088E592E069D58823C1F0609141
:100D9000730124E0629FC0011124FC01EC5AFE4F54
:100DA000238124FD02C0206101C02F7E2383FC012A
:100DB000EC5AFE4F238143E086E392E0A4D161E048
:100DC00088E592E04BD58823C1F06091730124E05F
:100DD000629FC0011124FC01EC5AFE4F238123FDC8
:100DE00002C0286001C0277F2383FC01EC5AFE4F1C
:100DF000238143E086E392E086D162E088E592E0D9
:100E00002DD5882309F475C06091730124E0629F99
:100E1000C0011124FC01EC5AFE4F238125FD02C0C4
:100E200020625AC02F7D58C066E088E592E00CD55C
:100E3000882309F45EC060E088E592E00FD588233E
:100E4000C1F06091730124E0629FC0011124FC0194
:100E5000EC5AFE4F238120FD02C0216001C02E7F8D
:100E60002383FC01EC5AFE4F238143E086E392E0AA
:100E70004AD161E088E592E0F1D48823C1F0609125
:100E8000730124E0629FC0011124FC01EC5AFE4F63
:100E9000238122FD02C0246001C02B7F2383FC013B
:100EA000EC5AFE4F238143E086E392E02CD162E0CE
:100EB00088E592E0D3D48823E1F06091730124E0C7
:100EC000629FC0011124FC01EC5AFE4F238121FDD9
:100ED00002C0226001C02D7F2383FC01EC5AFE4F2B
:100EE000238143E086E392E0DF91CF911F910F9140
:100EF0000AC1DF91CF911F910F9108950F931F9316
:100F000080914C01882321F184D7009148011091F0
:100F1000490120914A0130914B01601B710B820BFA
:100F2000930B6A3071058105910508F43FC010925A
:100F30004C016FD7609348017093490180934A0137
:100F400090934B0160E089E00E94271060E029C087
:100F500060D7009148011091490120914A013091D8
:100F60004B01601B710B820B930B009104011091DC
:100F7000050120E030E06017710782079307B0F0A9
:100F800081E080934C0145D76093480170934901FB
:100F900080934A0190934B0161E089E00E94271001
:100FA00061E08AE01F910F910C9427101F910F911F
:100FB00008950F931F93809153018823B1F029D78F
:100FC00000914F0110915001209151013091520137
:100FD000601B710B820B930B6431710581059105C8
:100FE00010F01092530167E007C0E0917301F0E048
:100FF000E459FE4F60816F5F88E592E01F910F9189
:1010000036C386E392E088D088E592E0EED361E0D3
:1010100070E080E090E039D766E088E592E01ED489
:10102000811133C066E088E592E022D481112DC0A1
:1010300039DD64E088E592E01BD4882389F0809153
:101040004D0181110DC025C08F5F808301C01082CA
:10105000E081F0E0EB5CFE4F408186E392E04FD010
:10106000A8DFB8DC80914D0181110CC066E088E5F5
:1010700092E0EAD3811106C064E088E592E0E4D30F
:10108000882389F0EBDBC2DD39CF88E592E062D2BC
:10109000CFCF60917301E62FF0E0E459FE4F8081DD
:1010A0008230A8F6D1CF7DDBEDCF13D7E7DAA9DF09
:1010B000FECF88E592E096C1CB010C940111CB01E3
:1010C000642F0C94091187E792E032C187E792E020
:1010D00081C1462F64E087E792E030C1462F68E087
:1010E00087E792E02BC1685D87E792E027C16E5CDD
:1010F00087E792E023C1645C87E792E01FC16A5BE7
:1011000087E792E01BC16C598AE0489F600D11246B
:10111000422F87E792E012C1EF92FF920F931F9345
:10112000CF93DF931F92CDB7DEB77C010AE010E0CA
:1011300087E792E014D1882309F4B6C087E792E0EC
:1011400043D1282F87E792E0298341D1482F298175
:10115000243049F138F42230D1F0F8F4213009F08C
:1011600045C008C0263059F120F1273071F12830F0
:10117000E9F531C0813029F087E792E049832DD12C
:101180004981D7011296ED91FC91139729C0D7019F
:101190001496ED91FC91159723C0D7011696ED9109
:1011A000FC9117971DC0D7011896ED91FC911997E6
:1011B00017C0D7011A96ED91FC911B9711C0D7016A
:1011C0001C96ED91FC911D970BC0D7011E96ED91D9
:1011D000FC911F9705C0D7015096ED91FC91519756
:1011E000309709F4A5CF842F0995A2CF822F8A507A
:1011F0008A3030F4D7015296ED91FC9153973BC061
:10120000822F84518A3030F4D7015496ED91FC91AD
:10121000559731C0822F8E518A3030F4D7015696BF
:10122000ED91FC91579727C0822F88528A3030F475
:10123000D7015896ED91FC9159971DC0822F82538A
:101240008A3030F4D7015A96ED91FC915B9713C028
:10125000822F8C538A3030F4D7015C96ED91FC914B
:101260005D9709C0822F86548A3058F4D7015E9664
:10127000ED91FC915F97309709F45ACF642F09954F
:1012800057CF243608F454CFD7019096ED91FC91B6
:101290009197309709F44CCF822F90E084569109B2
:1012A000B801F4D7099544CF0F90DF91CF911F91EA
:1012B0000F91FF90EF900895FC017383628308956E
:1012C000FC01758364830895FC0177836683089528
:1012D000FC01718760870895FC0173876287089518
:1012E000FC01758764870895FC01778766870895F8
:1012F000FC01738B628B0895FC01758B648B0895E0
:10130000FC01778B668B0895FC01718F608F0895C7
:10131000FC01738F628F0895FC01758F648F0895AF
:10132000FC01778F668F0895FC0171A360A3089577
:10133000AB0160E070E08AE792E0DFC3CF93C42F97
:101340008AE792E0693011F426D304C024D3C9306F
:1013500009F4CAE06C2F8AE792E0CF911CC3CF93C7
:10136000DF93EC018AE792E0B8D2892B39F18A81C8
:1013700081110EC08AE792E0DFD2888391E09A83E0
:10138000893031F48981893019F41A8218821982DE
:101390008A81813091F48AE792E09FD2892B71F0A3
:1013A0008AE792E0C9D289831A829881993041F400
:1013B000893031F41882198203C003C080E001C073
:1013C00081E0DF91CF910895FC0180810895FC01B7
:1013D0008181089549E069E0B1CFFC011282108259
:1013E0001182089522E0FC01218308952F923F92FB
:1013F0004F925F926F927F928F929F92AF92BF9225
:10140000CF92DF92EF92FF920F931F93CF93DF93D0
:10141000EC011F8682E2C82E81E0D82E7E0100E01A
:1014200010E066246A9493E0792E812C912C54016B
:101430008394F60181916F0187D5A301481B590B55
:10144000F70160897189CA01861B970B97FF03C05A
:101450009195819591092D8D21111FC0EE852E2F1B
:1014600030E0002E02C0359527950A94E2F720FF60
:1014700014C0813291058CF014012501002E04C0A6
:10148000220C331C441C551C0A94D2F7222D2095A3
:101490002E232E872F8522292F87298130E0281798
:1014A00039077CF4D501C401002E04C0880F991FB0
:1014B000AA1FBB1F0A94D2F72F85282B2F871A82C9
:1014C00014C08A818A3178F0D501C401002E04C08D
:1014D000880F991FAA1FBB1F0A94D2F780959F857A
:1014E00098239F8702C08F5F8A83F701778B668B73
:1014F000518B408B0F5F1F4FF2E0EF0EF11C03305A
:10150000110509F096CFDF91CF911F910F91FF90B8
:10151000EF90DF90CF90BF90AF909F908F907F9093
:101520006F905F904F903F902F900895FC018685BB
:1015300090E002C0959587956A95E2F781700895CD
:10154000FC01878590E002C0959587956A95E2F742
:1015500081700895FC012685276026870895262F2F
:1015600041E050E060E070E004C0440F551F661F8A
:10157000771F2A95D2F74095FC01268524232687DC
:101580000895FC01E60FF11DE60FF11D70968081B4
:1015900091810895FC01E60FF11DE60FF11D76968D
:1015A000808191810895EF92FF920F931F93CF93C3
:1015B000DF938C01FC01808165E2E62E61E0F62E6E
:1015C000C0E0D0E08823B1F0F801658570E00C2E12
:1015D00002C0759567950A94E2F76170772781E0FC
:1015E0006827F70181917F0132D52196C330D1055B
:1015F00059F715C0F801658570E00C2E02C075958D
:1016000067950A94E2F76170772781E06827F70110
:1016100081917F011CD52196C630D10559F7DF9104
:10162000CF911F910F91FF90EF900895FC01862FAD
:101630009585442369F041E050E060E070E004C02B
:10164000440F551F661F771F8A95D2F7492B0DC08F
:1016500041E050E060E070E004C0440F551F661F99
:10166000771F8A95D2F74095492345870895EF92D1
:10167000FF920F931F93CF93DF938C01E62FF0E03F
:10168000E65EFE4FE080C0E0D0E0F12CA7010C2E1A
:1016900002C0559547950A94E2F7417055276C2F83
:1016A0006D5FC801C3DF2196C330D10579F7DF91A3
:1016B000CF911F910F91FF90EF900895AF92BF923D
:1016C000CF92DF92EF92FF920F931F93CF93DF930E
:1016D000EC01EBE2AE2EE1E0BE2E00E010E0C12C0A
:1016E000D12C7601C394F50181915F01E6D42B8161
:1016F0003C81892B69F4D701C601002E04C0880FF4
:10170000991FAA1FBB1F0A94D2F7822B932B0EC0DE
:10171000D701C601002E04C0880F991FAA1FBB1F46
:101720000A94D2F780959095822393239C838B8390
:10173000D701C601002E04C0880F991FAA1FBB1F26
:101740000A94D2F79C01FC01E095F09569857A85B1
:101750006E237F237A8769874B855C854E235F23C1
:101760005C874B87AB81BC81002E02C0B595A795E5
:101770000A94E2F78D819E81A0FF1AC0AC01002E71
:1017800002C0559547950A94E2F740FD1BC0622BB5
:10179000732B7A87698716C0242B352B3C872B87C0
:1017A00014C00F5F1F4F0730110509F09CCF12C006
:1017B000BC01002E02C0759567950A94E2F760FDA2
:1017C000EBCF03C0822B932B02C08E239F239E83DB
:1017D0008D83E7CFDF91CF911F910F91FF90EF9015
:1017E000DF90CF90BF90AF900895CF93DF93EC013F
:1017F000FDDDCE0163DFCE01DF91CF91D4CE0F931B
:101800001F93CF93DF93EC010BE211E062E0F8014C
:1018100081918F01E4D3F1E002331F07B9F705E2AC
:1018200011E061E0F80181918F01D9D3F1E00B3231
:101830001F07B9F7CE018EDECE01D7DFCE01DF91D3
:10184000CF911F910F91D1CFFC018381948102C070
:10185000959587956A95E2F781700895FC018185D9
:10186000928502C0959587956A95E2F781700895F3
:10187000FC018385948502C0959587956A95E2F76A
:1018800081700895FC01A62F878190859C0102C07C
:10189000359527956A95E2F741E050E060E070E009
:1018A00004C0440F551F661F771FAA95D2F720FD6D
:1018B00003C0482B592B04C0409550954823592309
:1018C000508747830895FC018781908502C09595D4
:1018D00087956A95E2F781700895FC018485958566
:1018E000FC01E05CFF4F20813181FC01EE5BFF4F8A
:1018F00080819181281B390B2F733327C9010895EB
:10190000FC0184859585FC01E05CFF4F408151819D
:10191000FC01EE5BFF4F208131814217530741F0FC
:101920000190F081E02DE80FF91F208130E002C026
:101930002FEF3FEFC9010895FC0184859585FC01D7
:10194000E05CFF4F40815181FC01EE5BFF4F208145
:1019500031814217530781F0A081B181A80FB91FCF
:101960008C91208131812F5F3F4F2F73332731833B
:101970002083282F30E002C02FEF3FEFC9010895E8
:10198000FC0181A1882329F0A489B5898C9186FF67
:10199000FBCF11A20895CF93DF93FC0126853785F5
:1019A000D901A05CBF4F8D919C91119701968F73C7
:1019B0009927E901CE5BDF4F48815981841795074C
:1019C000D9F30D90BC91A02DA20FB31F6C93A685E7
:1019D000B785A05CBF4F11969C938E93A689B7895B
:1019E0002C9181E090E0078C02C0880F991F0A9427
:1019F000E2F7282B2C9381E081A30488F589E02D60
:101A000080818064808381E090E0DF91CF910895B0
:101A10001F920F920FB60F9211242F933F934F9363
:101A20008F939F93EF93FF938091C00082FD1CC022
:101A30004091C600809120039091210301968F73FD
:101A4000992720912203309123038217930771F085
:101A5000E0912003F0912103E052FD4F40839093E9
:101A600021038093200302C08091C600FF91EF9173
:101A70009F918F914F913F912F910F900FBE0F909B
:101A80001F9018951F920F920FB60F9211242F934B
:101A90003F938F939F93EF93FF932091DC023091BC
:101AA000DD028091DE029091DF022817390731F4C0
:101AB0008091C1008F7D8093C10014C0E091DE024F
:101AC000F091DF02E456FD4F20818091DE0290917B
:101AD000DF0201968F7399279093DF028093DE02D5
:101AE0002093C600FF91EF919F918F913F912F918D
:101AF0000F900FBE0F901F901895CF92DF92EF922C
:101B0000FF92CF93DF93EC016A017B01411581EED7
:101B1000580761057105F1F0EC89FD8981E090E0DD
:101B200008A002C0880F991F0A94E2F7808360E042
:101B300079E08DE390E0A7019601BBD321503109F4
:101B4000410951095695479537952795211580E10B
:101B5000380790F0EC89FD89108260E874E88EE126
:101B600090E0A7019601A5D32150310941095109FF
:101B70005695479537952795E889F9893083EA89FD
:101B8000FB89208319A2EE89FF89408181E090E0E2
:101B90009C010C8C02C0220F331F0A94E2F7422BE7
:101BA0004083EE89FF8940819C010D8C02C0220F89
:101BB000331F0A94E2F7422B4083EE89FF8940816C
:101BC0009C010E8C02C0220F331F0A94E2F7422BB5
:101BD0004083EE89FF8920810F8C02C0880F991FF6
:101BE0000A94E2F7809582238083DF91CF91FF9062
:101BF000EF90DF90CF90089510927D0210927C02BA
:101C000088EE93E0A0E0B0E080937E0290937F02A4
:101C1000A0938002B09381028CE391E090937B02C9
:101C200080937A0280EE92E09093870280938602FE
:101C30008CE992E0909389028093880285EC90E091
:101C400090938B0280938A0284EC90E090938D02B3
:101C500080938C0280EC90E090938F0280938E02B0
:101C600081EC90E0909391028093900282EC90E05E
:101C7000909393028093920286EC90E09093950269
:101C80008093940284E08093960283E0809397028D
:101C900087E08093980285E08093990281E08093A9
:101CA0009A020895CF92DF92EF92FF920F931F93C3
:101CB000CF93DF936C01EB017A01E60EF71E00E093
:101CC00010E00BC06991D601ED91FC910190F0817B
:101CD000E02DC6010995080F191FCE15DF0591F7F4
:101CE000C801DF91CF911F910F91FF90EF90DF908E
:101CF000CF9008954F925F926F927F92AF92BF9272
:101D0000CF92DF92EF92FF920F931F93CF93DF93C7
:101D1000CDB7DEB729013A01621B730B840B950B1B
:101D200029893A894B895C892A193B094C095D0943
:101D3000298B3A8B4B8B5C8B9B01AC0169897A892F
:101D40008B899C8974D2E418F50806091709A80143
:101D50009701D1D22A0D3B1D4C1D5D1DB901CA0151
:101D6000DF91CF911F910F91FF90EF90DF90CF9077
:101D7000BF90AF907F906F905F904F9008951F92AB
:101D80000F920FB60F9211242F933F938F939F932F
:101D9000AF93BF938091240390912503A0912603D4
:101DA000B091270330912C03232F2D5F2D3720F482
:101DB0000196A11DB11D05C0232F2A570296A11D12
:101DC000B11D20932C038093240390932503A093AB
:101DD0002603B09327038091280390912903A091B3
:101DE0002A03B0912B030196A11DB11D80932803F6
:101DF00090932903A0932A03B0932B03BF91AF9133
:101E00009F918F913F912F910F900FBE0F901F9038
:101E100018950F931F938FB7F89400912403109196
:101E2000250320912603309127038FBFB801C901F4
:101E30001F910F9108950F931F939FB7F8940091EE
:101E400028031091290320912A0330912B0386B592
:101E5000A89B06C08F3F21F00F5F1F4F2F4F3F4FB2
:101E60009FBF322F212F102F0027080F111D211D7A
:101E7000311D42E0000F111F221F331F4A95D1F779
:101E8000B801C9011F910F910895CF92DF92EF928F
:101E9000FF92CF93DF936B017C01CDDFEB010DC08F
:101EA000CADF6C1B7D0B683E734038F081E0C81AB6
:101EB000D108E108F108C851DC4FC114D104E10494
:101EC000F10471F7DF91CF91FF90EF90DF90CF9009
:101ED0000895789484B5826084BD84B5816084BDA2
:101EE00085B5826085BD85B5816085BDEEE6F0E093
:101EF000808181608083E1E8F0E0108280818260EF
:101F00008083808181608083E0E8F0E0808181606F
:101F10008083E1EBF0E0808184608083E0EBF0E09F
:101F2000808181608083EAE7F0E080818460808343
:101F300080818260808380818160808380818068ED
:101F400080831092C10008958E3008F08E50877003
:101F50002091320140E4249F90011124822B809330
:101F60007C0080917A00806480937A0080917A006E
:101F700086FDFCCF2091780030917900932F80E08E
:101F8000AC01422B9A01C9010895833069F028F40D
:101F90008130A1F0823011F514C08630B1F0873065
:101FA000C1F08430D9F404C0809180008F7703C0E1
:101FB000809180008F7D80938000089584B58F7715
:101FC00002C084B58F7D84BD08958091B0008F7765
:101FD00003C08091B0008F7D8093B0000895CF93AF
:101FE000DF9390E0FC01E458FF4F4491FC01E0577F
:101FF000FF4F8491882341F190E0880F991FFC01E5
:10200000E854FF4F25913491D90182559F4FFC012F
:1020100085919491C82FD92F9FB7F8948C91611115
:1020200006C0409584238C938881842308C0623045
:1020300041F4242F209582238C938881842B8883DC
:1020400002C0842B8C939FBFDF91CF9108950F9393
:102050001F93CF93DF931F92CDB7DEB7282F30E0C9
:10206000F901E859FF4F8491F901E458FF4F1491A9
:10207000F901E057FF4F04910023C9F0882319F0BC
:10208000698383DF6981E02FF0E0EE0FFF1FE255E7
:10209000FF4F85919491DC019FB7F8948C91611169
:1020A00003C01095812301C0812B8C939FBF0F909B
:1020B000DF91CF911F910F910895CF93DF93282F38
:1020C00030E0F901E859FF4F8491F901E458FF4FDE
:1020D000D491F901E057FF4FC491CC2381F08111D5
:1020E00054DFEC2FF0E0EE0FFF1FEC55FF4F859112
:1020F0009491DC018C918D2321E030E011F420E0FB
:1021000030E0C901DF91CF9108958770806480939A
:102110007C00EAE7F0E08081806480830895CF93BB
:10212000DF931F92CDB7DEB780913F0390914003BC
:102130008F3F2FEF920761F0FC01E75CFC4F20819D
:10214000298301979093400380933F03898101C0C5
:102150008FEF80933301809133018F3F19F080918D
:102160003301D3DF0F90DF91CF910895EAE7F0E0DC
:102170008081806480830895E091330180917800AC
:1021800090917900EE0FFF0BE35DFC4F918380830C
:1021900008951F920F920FB60F9211242F933F9321
:1021A0004F935F936F937F938F939F93AF93BF935F
:1021B000EF93FF9380913401882321F0D7DF1092B1
:1021C000340105C0D9DFABDF81E080933401FF919A
:1021D000EF91BF91AF919F918F917F916F915F919F
:1021E0004F913F912F910F900FBE0F901F90189518
:1021F0008FEF9FEF9093400380933F030895F894EF
:10220000B1C0F999FECF92BD81BDF89A992780B5EA
:102210000895262FF999FECF1FBA92BD81BD20BD2A
:102220000FB6F894FA9AF99A0FBE01960895DB0159
:102230008F939F937BD0BF91AF91A29F800D911DF3
:10224000A39F900DB29F900D11240895991B79E0E2
:1022500004C0991F961708F0961B881F7A95C9F736
:1022600080950895AA1BBB1B51E107C0AA1FBB1F85
:10227000A617B70710F0A61BB70B881F991F5A9512
:10228000A9F780959095BC01CD01089597FB072E85
:1022900016F4009406D077FD08D0E4DF07FC05D0E3
:1022A0003EF4909581959F4F0895709561957F4F6D
:1022B0000895A1E21A2EAA1BBB1BFD010DC0AA1F87
:1022C000BB1FEE1FFF1FA217B307E407F50720F09F
:1022D000A21BB30BE40BF50B661F771F881F991F1A
:1022E0001A9469F760957095809590959B01AC0163
:1022F000BD01CF010895052E97FB16F4009406D07A
:1023000057FD0CD0D6DF07FC09D07EF49095809560
:10231000709561957F4F8F4F9F4F089550954095D1
:10232000309521953F4F4F4F5F4F08950FD0A59F98
:10233000900DB49F900DA49F800D911D11240895C0
:10234000EE0FFF1F0590F491E02D0994A29FB001BC
:10235000B39FC001A39F01D0B29F700D811D1124B6
:08236000911D0895F894FFCFD0
:1023680001000000640000003F007F00BF00FF0084
:102378000A006400FA00E803D0070001020403051C
:1023880006070F1210020607050304080D0C110BAF
:10239800130E01FF0104050600000000CB0C520ECD
:0823A8006D0C9C0C800CC00CB4
:00000001FF
